S01D000062696E2F6F70656E626C745F73746D3332663734362E737265638C
S31508000000000005203503000885030008850300085D
S315080000108503000885030008850300080000000022
S315080000200000000000000000000000008503000832
S31508000030850300080000000085030008A94500089C
S315080000408503000885030008850300088503000862
S315080000508503000885030008850300088503000852
S315080000608503000885030008850300088503000842
S315080000708503000885030008850300088503000832
S315080000808503000885030008850300088503000822
S315080000908503000885030008850300088503000812
S315080000A08503000885030008850300088503000802
S315080000B085030008850300088503000885030008F2
S315080000C085030008850300088503000885030008E2
S315080000D085030008850300088503000885030008D2
S315080000E085030008850300088503000885030008C2
S315080000F085030008850300088503000885030008B2
S3150800010085030008850300088503000885030008A1
S315080001108503000885030008850300088503000891
S315080001208503000885030008850300088503000881
S315080001308503000885030008850300088503000871
S315080001408503000885030008850300088503000861
S315080001508503000885030008850300088503000851
S315080001608503000885030008850300088503000841
S3150800017085030008850300088503000800000000C1
S315080001808503000885030008850300088503000821
S315080001908503000885030008850300088503000811
S315080001A08503000885030008850300088503000801
S315080001B085030008850300088503000885030008F1
S30D080001C0850300088503000809
S315080001C810B5054C237833B9044B13B10448AFF37B
S315080001D800800123237010BDEC04002000000000F5
S315080001E8C050000808B5034B1BB103490348AFF3D1
S315080001F8008008BD00000000F0040020C050000878
S3150800020870B50D4E0D4D761BB61006D00024013478
S3150800021855F8043B9847A642F9D1094E094D761B6D
S3150800022804F04AFFB61006D00024013455F8043BFA
S315080002389847A642F9D170BD4452000844520008AE
S315080002484C52000844520008024B13B1024800F009
S3150800025805B870470000000071020008002301462F
S315080002681A46184600F01EB838B50A4C0A4D641BDB
S31508000278A4100AD004F18043013B05EB8305013C31
S3150800028855F804399847002CF9D1BDE8384004F0E8
S3150800029819BF00BF505200084C520008704700BFEB
S315080002A8704700BF2DE9F0411E4C05462068904668
S315080002B81F460E46FFF7F2FF1B4B1A68D2F848315D
S315080002C833B35A6820681F2A27DC4DB9911C0132B6
S315080002D85A6043F82160FFF7E3FF0020BDE8F08184
S315080002E803EB82010124C1F8888004FA02FED3F8D8
S315080002F88841022D44EA0E0CC3F888C1C1F8087172
S31508000308E4D1D3F88C114EEA0104C3F88C41DDE731
S3150800031802F5A673C2F84831D3E7FFF7C1FF4FF0D5
S31508000328FF30DBE728040020D8500008DFF834D06F
S31508000338002103E00C4B5B58435004310B480C4B27
S3150800034842189A42F6D30B4A02E0002342F8043BC5
S31508000358094B9A42F9D300F007FDFFF751FF03F05E
S315080003683DFB704700000520505200080000002099
S31508000378EC040020EC0400208C140020FEE710B5DD
S3150800038813460222C0F86C22C36103620A4600219A
S3150800039803F0BAFD002010BD08B513460A46002129
S315080003A803F0B2FD002008BD08B513460A46002129
S315080003B803F0B2FD002008BD08B50423C0F86C3266
S315080003C800231A46194603F09FFD002008BD08B504
S315080003D80523C0F86C3200231A46194603F09CFD1B
S315080003E8002008BD002302781AB10133DBB20130B8
S315080003F8F9E71846704708B54B88012B00D008BDA1
S31508000408C0F87C32FFF7D8FFF9E70B7803704B780A
S3150800041843708B78CA7803EB022343800B794A79B1
S3150800042803EB022383808B79CA7903EB0223C38003
S31508000438704710B50446802103F04EFD002120467A
S3150800044803F04AFD10BD30B583B005460C464A8808
S31508000458130A013B062B00F28480DFE803F0041632
S315080004682A8282667300D0F888321B680DF1060165
S31508000478007C9847BDF8062012B1E388002B74D192
S31508000488E388002B7BD003B030BD037C43B9D0F892
S315080004988C329B6A0DF10600984702234370E9E7F8
S315080004A8D0F88C32DB6A0DF10600984702234370B0
S315080004B8E0E7D2B2052A34D8DFE802F0030B131BAB
S315080004C8232BD0F888325B680DF10601007C984723
S315080004D8D0E7D0F888329B680DF10601007C98476A
S315080004E8C8E7D0F88832DB680DF10601007C984722
S315080004F8C0E7D0F888321B690DF10601007C9847D9
S31508000508B8E7D0F888325B690DF10601007C984790
S31508000518B0E7D0F888329B690DF10601007C984748
S31508000528A8E72146FFF785FFADE7037C33B9D0F87E
S315080005388C325B6B0DF1060098479BE72146FFF75F
S3150800054878FFA0E7037C43B9D0F88C321B6B0DF112
S3150800055806009847072343708CE72146FFF769FF8B
S3150800056891E72146FFF765FF8DE79A4228BF1A46A5
S31508000578ADF8062001462846FFF701FF80E728461A
S31508000588FFF71AFF7FE738B504468B88F3B9CB8897
S31508000598E3B94B887F2B19D803F07F0590F8743296
S315080005A8032B0CD080F87652294603F0A5FC204682
S315080005B8FFF702FF35B1022384F8743209E0FFF722
S315080005C838FF06E0012384F8743202E02046FFF774
S315080005D830FF38BD38B504460D468978284B19705A
S315080005E801290ED890F87432022B0ED0032B21D08D
S315080005F82946FFF71EFF224B1978204600F070FAA5
S3150800060802E02946FFF715FF38BD81B1416003238B
S3150800061880F8743200F057FA022803D02046FFF70C
S31508000628CBFEF1E729462046FFF703FFECE7FFF77D
S31508000638C3FEE9E789B1436899421DD0D9B200F0EB
S315080006484FFA0F4B19786160204600F03CFA0228E9
S315080006580DD02046FFF7B0FED6E7022380F874329D
S31508000668416000F03DFA2046FFF7A6FECCE729468A
S315080006782046FFF7DEFEC7E7FFF79EFEC4E700BF82
S315080006880805002008B5CB88012B0CD190F87432E0
S315080006985AB29AB1022B09D9032B0FD10122011D8F
S315080006A8FFF76DFE01E0FFF7C4FE08BD014600230B
S315080006B841F8083F0122FFF762FEF6E7FFF7B9FEA1
S315080006C8F3E708B590F87432013B022B12D8CB88A9
S315080006D8022B0CD10123C360D0F87C320BB103235B
S315080006E8C360022200F10C01FFF749FE08BDFFF7B7
S315080006F8A0FEFBE7FFF79DFEF8E708B590F8743209
S31508000708013B022B09D84B88012B00D008BD0023D2
S31508000718C0F87C32FFF750FEF8E7FFF78AFEF5E7E0
S3150800072808B50B7803F06003202B05D0402B03D0BF
S3150800073843B1FFF77EFE03E0D0F88C329B689847F2
S31508000748002008BD4B78092B1BD8DFE803F01117E2
S315080007581A141A08051A0E0BFFF775FEF0E7FFF7C5
S3150800076812FFEDE7FFF736FFEAE7FFF78BFFE7E744
S31508000778FFF7A7FFE4E7FFF73EFEE1E7FFF7BDFF50
S31508000788DEE7FFF756FEDBE738B505460C460B7875
S3150800079803F06003202B06D0402B04D01BB1FFF7CB
S315080007A848FE002038BD95F87432013B022B16D84E
S315080007B82379012B0ED8D5F88C329B682146284612
S315080007C89847E388002BECD10028EAD12846FFF79A
S315080007D8F3FDE6E721462846FFF72BFEE1E7214623
S315080007E82846FFF726FEDCE738B504468A880B78DC
S315080007F803F06003202B08D0D0B2402B05D05BB19C
S315080008082046FFF716FE002005E0D4F88C329B68D0
S3150800081820469847002038BD202B13D04B78012B4B
S3150800082843D05DB2002D73D0032B40F0F58094F8C1
S315080008387432022B0CD0032B21D02046FFF7F9FD82
S315080008480020E8E7D4F88C329B6820469847E2E708
S31508000858B0F1800318BF0123002808BF00234BB155
S315080008680146204603F038FB8021204603F034FB76
S315080008780020D0E72046FFF7DCFD0020CBE74B88B1
S315080008884BB9B0F1800318BF0123002808BF00231D
S315080008980BB1CB8823B12046FFF78EFD0020BAE7B7
S315080008A80146204603F018FBF5E794F87432022B44
S315080008B806D0032B1BD02046FFF7BBFD0020AAE76E
S315080008C8B0F1800318BF0123002808BF00234BB1E5
S315080008D80146204603F000FB8021204603F0FCFA77
S315080008E8002098E72046FFF7A4FD002093E74B88E9
S315080008F8002B40F0968010F07F0F04D12046FFF7B2
S315080009085BFD002087E70146204603F0EDFAF5E788
S3150800091894F87432022B06D0032B2ED02046FFF704
S3150800092888FD002077E7B0F1800318BF0123002867
S3150800093808BF002393B912F0800F14D100F07F0086
S3150800094800EB8000830003F5A073E11800250D600D
S3150800095802222046FFF713FD28465CE72046FFF7E4
S3150800096868FD002057E700F07F0000EB8000830051
S3150800097803F1100121440431E8E752B2002A23DBC7
S3150800098800F00F0303EB83039D002544D5F8443193
S3150800099843B3002A2BDB00F07F0202EB82029300A6
S315080009A803F5A073E518802814BF0023012300283F
S315080009B808BF01232BB300232B60022229462046B1
S315080009C8FFF7DDFC002026E700F00F0303EB83039F
S315080009D89D002544AB69002BDBD12046FFF729FD8E
S315080009E8002018E72046FFF724FD002013E700F04B
S315080009F87F0202EB8202930003F1100525440435B1
S31508000A08D1E70146204603F013FA10B101232B60FB
S31508000A18D3E700232B60D0E72046FFF70AFD00201E
S31508000A28F9E60020F7E6C0B170B50D461646044645
S31508000A38FFF7D8FC013040003080287003236B701C
S31508000A480223217841B101345A1CD2B2E95402333F
S31508000A58DBB20021A954F4E770BD704798B108B510
S31508000A680346D0F88C0210B10020C3F88C0209B1ED
S31508000A78C3F888121846012380F87432027003F006
S31508000A889DF9002008BD0220704710B504460123C9
S31508000A9880F87432D0F88C325B680179984720461A
S31508000AA803F0FFF9204603F0ECF9002010BD19B150
S31508000AB8C0F88C12002070470220704708B503F06A
S31508000AC8E8F9002008BD08B5D0F88C3233B11B68A0
S31508000AD8984708B9002008BD0220FCE70220FAE773
S31508000AE808B5D0F88C325B689847002008BD38B539
S31508000AF8044600F520752846FFF787FC0123C4F845
S31508000B086C32B4F88632C4F8703294F8801201F060
S31508000B181F03012B0FD05AB23AB1022B10D001F09D
S31508000B288001204603F0D8F903E029462046FFF756
S31508000B38F7FD002038BD29462046FFF725FEF8E7C9
S31508000B4829462046FFF750FEF3E738B50446A9BB01
S31508000B581046D4F86C32032B03D0052B25D0002079
S31508000B6838E0D4F84C31D4F8502193420DD99B1A61
S31508000B78C4F84C319A4206D99AB201462046FFF77C
S31508000B8813FC002026E092B2F7E7D4F88C321B69EA
S31508000B981BB194F87422032A04D02046FFF70CFCEC
S31508000BA8002017E020469847F7E70025C4F86C5256
S31508000BB82946204603F090F928460BE00A46D0F85D
S31508000BC88C329B693BB190F87412032905D11146FA
S31508000BD89847002038BD0220FCE70220FAE710B53E
S31508000BE80446002956D11046D4F86C32022B09D08F
S31508000BF8002B18BF042B44D094F87832012B45D023
S31508000C08002010BD236A626A93421BD8E169B1FBCA
S31508000C18F2F302FB13132BB98A4203D8D4F87032BD
S31508000C2899421DD3D4F88C32DB681BB194F8742228
S31508000C38032A23D08021204603F04EF92046FFF7E1
S31508000C48C6FBD9E79A1A226292B201462046FFF7EE
S31508000C58A3FB00231A461946204603F05DF9CBE79D
S31508000C68002211462046FFF797FB0021C4F87012A8
S31508000C780B460A46204603F04FF9BDE72046984733
S31508000C88D8E78021204603F027F9B5E7002084F83D
S31508000C987802B6E70A46D0F88C325B693BB190F819
S31508000CA87412032905D1114698470020A9E702209E
S31508000CB8A7E70220A5E770B5044640230022114697
S31508000CC803F0F7F80125C4F844514026C4F85061E2
S31508000CD8334600228021204603F0EBF8A5616662B8
S31508000CE884F874520023C4F86C326360C4F87C3202
S31508000CF8D4F890322BB1D4F88C325B6800212046A0
S31508000D089847002070BD01740020704790F8743227
S31508000D1880F87532042380F874320020704790F8FA
S31508000D28753280F874320020704708B590F8743226
S31508000D38032B01D0002008BDD0F88C32DB69002BC4
S31508000D48F8D09847F6E7002070470020704700203B
S31508000D58704708B5012280F87422D0F88C225268A8
S31508000D6801799047002008BD10B40F4AD2F8883098
S31508000D7843F47003C2F888300C4B196841F0010136
S31508000D881960002098601C680949214019600949BA
S31508000D985960196821F480211960D8604FF00063FA
S31508000DA893605DF8044B704700ED00E00038024098
S31508000DB8FFFFF6FE1030002410B5094B4FF0FF323E
S31508000DC81A6200241C625A625C621A611C615A61C2
S31508000DD85C619A619C6102F0AFFE204610BD00BFB7
S31508000DE80038024010B504460E4B18784FF47A734B
S31508000DF8B3FBF0F30C4A1068B0FBF3F001F054FEAD
S31508000E0868B90F2C01D901200AE0002221464FF0C3
S31508000E18FF3001F017FE054B1C60002000E001209A
S31508000E2810BD00BF300400202C0400203404002024
S31508000E3808B5032001F0F4FD0020FFF7D3FF02F000
S31508000E48D5FD002008BD000038B5044603F0A4FB0C
S31508000E580546B4F1FF3F02D0044B1B781C4403F047
S31508000E689BFB401BA042FAD338BD00BF30040020C4
S31508000E782DE9F04782B0D0F80080CA00521A9300CC
S31508000E8803445A6D1B6D9A4255D8C1469B1AC1EB45
S31508000E98C104A2000244526C9A4200D31A460C4670
S31508000EA8074602F1030A4FEA9A0A15E006F1030A09
S31508000EB84FEA9A0AE3001B1B9D003D44A96C3B7C3C
S31508000EC80093B3B2E2B2404602F024F9AB6C33445D
S31508000ED8AB646B6D1E446E6509EB441303F510632A
S31508000EE89B699BB2534512D3E3001B1B9A003A44ED
S31508000EF8516D136D99420AD24BB15B1AC4EBC40102
S31508000F088A003A44566C9E42D0D31E46CEE7E30082
S31508000F181B1B980007443A6D7B6D9A420FD804F05C
S31508000F280F040123A340D8F8344824EA0304C8F870
S31508000F383448002000E0012002B0BDE8F087002010
S31508000F48FAE77047F0B58BB0002800F08A800446A7
S31508000F5890F8BD33F3B1032384F8BD33206801F054
S31508000F6891FE254655F8107B6E460FCD0FC60FCD58
S31508000F780FC695E8030086E80300231D0ECB3846FE
S31508000F8801F0C6FD58B1022384F8BD330125284669
S31508000F980BB0F0BD80F8BC33FFF7D3FFDBE70021C1
S31508000FA8206801F075FE00236568AB4216D2D900A1
S31508000FB8C81A82002244012082F83D0082F83C3093
S31508000FC8A2F84230002082F83F0050649064CA1A9A
S31508000FD89100214408650133DBB2E5E700239D4209
S31508000FE816D9D800C11A8A002244002182F8FD11B0
S31508000FF882F8FC3182F8FF11C2F80412C2F8081206
S31508001008C21A90002044C0F810120133DBB2E6E792
S31508001018254655F8107B6E460FCD0FC60FCD0FC661
S3150800102895E8030086E80300231D0ECB384601F031
S3150800103875FE054660B9002384F83830012384F81C
S31508001048BD33636A012B08D0206802F018FA9EE7B8
S31508001058022384F8BD33012599E7204602F04EFBA2
S31508001068F2E7012593E7704790F8BC33012B0ED0B9
S3150800107810B50446012380F8BC33006802F0F3F97A
S31508001088206801F0F9FD002084F8BC0310BD022091
S31508001098704738B590F8BC33012B18D0044601239D
S315080010A880F8BC33006801F0EDFD206802F0A7F966
S315080010B8054628B1002384F8BC330125284638BDDF
S315080010C8206802F0DCF9002384F8BC33F6E7022529
S315080010D8F4E768B110B50446032380F8BD33FFF773
S315080010E8D8FF2046FFF7BFFF002084F8BD0310BDD0
S315080010F80120704770B505460E460368196C03EB60
S31508001108461303F53064A3680269012A09D0354AEB
S31508001118914261D113F4004F54D04FF40043A360B1
S315080011285DE013F0080F14D02F4A914205D913F43D
S31508001138004F02D04FF40043A360284602F0BAFDD8
S3150800114805F571720121286802F0F6F90823A360EB
S3150800115845E013F0200F02D02023A3603FE013F0E8
S31508001168280F3CD1204A914206D913F4004F03D0E0
S315080011784FF40043A36032E0F200921B93002B441D
S31508001188D3F804222169C1F31201521AC3F81422AA
S31508001198D3F80412D3F808220A44C3F80822F1B28D
S315080011A8284602F08FFDD6B9C6EBC606B3002B440F
S315080011B8D3F810329BB905F571720121286802F037
S315080011C8BBF90CE013F0200F01D02023A360F1B27D
S315080011D8284602F077FD02E0F1B202F073FD00201E
S315080011E870BD00BF0A31544F0A30544F38B504460B
S315080011F803681D6C03EB411101F530618A680369C0
S31508001208012B0DD0124B9D4214D0204602F052FDF8
S31508001218104B9D4202D92369012B12D0002038BDF4
S315080012280C4B9D42F1D912F4004FEED04FF400430F
S315080012388B60EAE712F4004FE7D04FF400438B605F
S31508001248E3E704F571720121206802F075F9E5E70C
S315080012580A31544F0A30544F2DE9F84F04460568A9
S31508001268284602F049F908B1BDE8F88FA8460746A6
S31508001278206802F010F90028F6D0206802F00BF969
S3150800128810F0020F04D02268536903F00203536171
S31508001298206802F000F910F4002F40F092803E46CC
S315080012A8206802F0F8F810F4802F40F0DC802068F7
S315080012B802F0F1F80028C0F24A81206802F0EBF83B
S315080012C810F4006F0AD0D5F8083813F0010F40F06B
S315080012D858812268536903F400635361206802F051
S315080012E8DAF810F0006F15D02268536903F0006326
S315080012F8536194F8F433002B40F04781012184F8B0
S31508001308F41323685B6DC3F38303C4F8F8332046E4
S3150800131802F008FA206802F0BEF810F4805F40F080
S315080013283881206802F0B7F810F4005F40F08A8127
S31508001338206802F0B0F810F0100F14D022689369EC
S3150800134823F0100393612F6A07F00F08C7F3434386
S31508001358022B00F08F81062B00F0AD812268936975
S3150800136843F010039361206802F095F810F0080F0F
S3150800137840F0B581206802F08EF810F4801F40F01E
S31508001388B781206802F087F810F4001F40F0BA8188
S31508001398206802F080F810F0804F40F0BD81206880
S315080013A802F079F810F0040F3FF45EAF23685D6821
S315080013B815F0040F40F0B981226853682B4353602F
S315080013C852E7206802F06BF881463E4624E008EBAF
S315080013D846130122C3F8082B31462046FFF78AFE32
S315080013E829E031462046FFF701FF08EB4613082295
S315080013F8C3F8082B22E008EB46132022C3F8082B6B
S315080014081AF4005F05D008EB46134FF40052C3F8E8
S31508001418082B01364FEA5909B9F1000F3FF440AFD6
S3150800142819F0010FF5D0F1B2206802F048F88246A3
S3150800143810F0010FCBD11AF0080FD2D11AF0100FFD
S3150800144804D008EB46131022C3F8082B1AF0200F0D
S31508001458D6D02369012BCED104F5717201212068F3
S3150800146802F06AF8C7E7206802F021F881463E4686
S315080014782EE0F200921B93002344596C9A6C0A4496
S315080014889A6448E01AF0080F04D008EB46130822B5
S31508001498C3F808291AF0100F04D008EB46131022CF
S315080014A8C3F808291AF0400F04D008EB461340225F
S315080014B8C3F808291AF0020F04D008EB46130222CB
S315080014C8C3F808291AF0800F3CD101364FEA5909A2
S315080014D8B9F1000F3FF4EBAE19F0010FF5D05FFA3A
S315080014E886FB5946206801F0F3FF824610F0010F83
S315080014F8C8D006F00F03012101FA03F2D8F83438E8
S3150800150823EA0203C8F8343808EB4613C3F808195F
S3150800151823698B42ADD05946204602F0DFFB236982
S31508001528012BAFD1002EADD1C6EBC60293002344DA
S315080015381B6D002BA6D104F571720121206801F0F4
S31508001548FBFF9FE731462046FFF792FCBDE7D5F833
S31508001558043823F00103C5F8043894F8F433012B4A
S3150800156808D0204602F000FC2268536903F00043BD
S315080015785361A2E6002184F8F413204602F0D2F853
S31508001588F2E7204602F0D6FBA3E6204602F0D2FB95
S31508001598C0E605F50069D9F8043023F00103C9F84F
S315080015A804301021206801F08BFB14E008EB471380
S315080015B84FF67F31C3F80819D3F8002922F4001228
S315080015C8C3F80029C3F8081BD3F8002B22F4001225
S315080015D8C3F8002B01376368BB42E7D8D9F81C3033
S315080015E843F00113C9F81C30236BEBB1D9F88430E2
S315080015F843F00B03C9F88430D9F8443043F00B0399
S31508001608C9F84430D5F8003823F4FE63C5F800381D
S3150800161804F57172217C206801F08EFF22685369EF
S3150800162803F4805353617CE6D9F8142042F22B035D
S315080016381343C9F81430D9F8103043F00B03C9F826
S315080016481030DFE7206801F05BFF206801F03EFCF8
S31508001658E060276800F06EFC227B0146384601F0F8
S3150800166895FA204602F04CFB2268536903F40053A6
S3150800167853615DE647F6F0731F423FF46FAE3F09C4
S315080016884FEAC80AAAEB08034FEA8309A144C7F335
S315080016980A02D9F80812284601F042FEC7F30A07D3
S315080016A8D9F808323B44C9F80832D9F814321F4425
S315080016B8C9F8147252E6082204F57171284601F031
S315080016C82FFEC7F30A174FEAC803A3EB08018A00D7
S315080016D82244D2F814321F44C2F814723EE6204651
S315080016E802F007FB2268536903F00803536141E6D1
S315080016F8F1B2204602F047FB2268536903F48013C7
S3150800170853613EE6F1B2204602F037FB2268536978
S3150800171803F4001353613BE6204602F03AFB2268BD
S31508001728536903F08043536139E6204602F03BFBD0
S3150800173842E690F8BC33012B0BD010B504460123BA
S3150800174880F8BC33006801F08EFE002084F8BC03DC
S3150800175810BD0220704790F8BC33012B0BD010B58A
S315080017680446012380F8BC33006801F088FE00208F
S3150800177884F8BC0310BD0220704790F8BC33012BCF
S315080017880DD010B50446012380F8BC3380F838100C
S31508001798006801F058FE002084F8BC0310BD02203A
S315080017A87047F8B511F0800F27D101F00F05EE0044
S315080017B8771BBC00274604F5FC7404440434074424
S315080017C8002587F8FD5101F00F012170A260E3702A
S315080017D8627802B1E180022B1ED090F8BC33012B47
S315080017E81DD00546012380F8BC332146006801F060
S315080017F87DFB002085F8BC03F8BD01F00F06F5004F
S31508001808AF1BBC0027463834044404343E46064415
S31508001818012586F83D50D6E700232371DDE7022027
S31508001828EAE738B511F0800F20D101F00F04E2007D
S31508001838151BAB001D4603F5FC7303440433054426
S31508001848002285F8FD2101F00F01197090F8BC23D4
S31508001858012A1AD00446012280F8BC2319460068D2
S3150800186801F08CFB002084F8BC0338BD01F00F0496
S31508001878E200151BAB001D463833034404332C46D7
S315080018880444012284F83D20DDE70220EDE770B51F
S3150800189801F00F05EE00711B8C0004F5FC74044476
S315080018A8211D761BB4000444C4F80822C4F8103273
S315080018B80023C4F8143284F8FD3184F8FC5103690E
S315080018C8012B06D065B9DAB2006801F09FFB002043
S315080018D870BDC5EBC506B4000444C4F80C22F1E78C
S315080018E8DAB2006801F02AFCF1E701F00F01C1EB52
S315080018F8C1018B001844D0F81402704770B501F07E
S315080019080F05EE00711B8C0038340444211D761B24
S31508001918B4000444A264236500236365012384F89C
S315080019283D3084F83C500369012B06D05DB9DAB21C
S31508001938006801F06BFB002070BDC5EBC506B40056
S315080019480444E264F2E7DAB2006801F0F7FBF2E76A
S3150800195838B501F00F0543689D4236D811F0800F57
S3150800196820D1CA00541AA3001C4603F5FC73034485
S31508001978043322460244002182F8FD1101229A7096
S315080019881D7090F8BC23012A21D00446012280F84C
S31508001998BC231946006801F0D7FC7DB1002084F8FD
S315080019A8BC0338BDEA00511B8B001946383303447B
S315080019B804330144012281F83D20DFE704F57172FA
S315080019C8217C206801F0B8FDE8E70120E9E7022054
S315080019D8E7E710B501F00F0443689C422CD811F0CC
S315080019E8800F1DD1E3001A1B91000A4601F5FC7108
S315080019F8014404310244002382F8FD3100238B7028
S31508001A080C7090F8BC33012B18D00446012380F8D3
S31508001A18BC33006801F0C5FC002084F8BC0310BD7F
S31508001A28E3001A1B91000A4638310144043102447E
S31508001A38012382F83D30E1E70120F0E70220EEE7CE
S31508001A48534B98421FD0534B984228D0524B984232
S31508001A5831D0524B98423AD0514B984243D0514BC9
S31508001A6898424CD0504B984255D0504B98425ED02D
S31508001A784F4B984267D04F4B984270D04E4B98427E
S31508001A8879D00120704703F560531A6942F00102BC
S31508001A981A611A6922F001021A610020704703F5D3
S31508001AA850531A6942F002021A611A6922F00202B0
S31508001AB81A610020704703F540531A6942F0040278
S31508001AC81A611A6922F004021A610020704703F5A0
S31508001AD830531A6942F008021A611A6922F0080294
S31508001AE81A610020704703F520531A6942F010025C
S31508001AF81A611A6922F010021A610020704703F564
S31508001B0810531A6942F020021A611A6922F0200253
S31508001B181A610020704703F500531A6942F040021B
S31508001B281A611A6922F040021A610020704703F503
S31508001B38E0531A6942F080021A611A6922F0800293
S31508001B481A610020704703F5C0531A6942F4807277
S31508001B581A611A6922F480721A610020704703F51F
S31508001B68A0531A6942F400721A611A6922F40072BB
S31508001B781A610020704703F580531A6942F4806297
S31508001B881A611A6922F480621A610020704700BF38
S31508001B98000002400004024000080240000C02400F
S31508001BA8001002400014024000180240001C0240BF
S31508001BB8002002400024024000280240F0B40C68C5
S31508001BC894FAA4F4B4FA84F42CE08E68826893FA3A
S31508001BD8A3F5B5FA85F56D0007FA05F522EA0502B3
S31508001BE893FAA3F5B5FA85F56D0006FA05F52A43BD
S31508001BF882600E69C26893FAA3F5B5FA85F56D0091
S31508001C08032707FA05F522EA050293FAA3F5B5FAB2
S31508001C1885F56D0006FA05F52A43C2604A68022A60
S31508001C2822D001340B6833FA04F250D00122A240BC
S31508001C381340F6D04E68026893FAA3F5B5FA85F507
S31508001C486D00032707FA05F522EA050293FAA3F5B4
S31508001C58B5FA85F56D0006FA05F52A4302604A685D
S31508001C68013A012AC5D8B0E793FAA3F2B2FA82F282
S31508001C78072A15D84D69026A93FAA3F6B6FA86F6BC
S31508001C88B6000F2707FA06F622EA060293FAA3F31E
S31508001C98B3FA83F39B0005FA03F313430362C0E719
S31508001CA84A69456A1B0A93FAA3F6B6FA86F6B6008F
S31508001CB80F2707FA06F625EA060593FAA3F3B3FAF1
S31508001CC883F39B0002FA03F32B434362A9E74A68A6
S31508001CD8013A012A02D90020F0BC7047C96842684F
S31508001CE822EA030201FB03F313434360F3E7000008
S31508001CF810B40A490C6924F440740C610C6944F45C
S31508001D0840740C610C6944F001040C61026043607C
S31508001D18BFF34F8F5DF8044B704700BF003C024085
S31508001D28084B1A6922F440721A611A6942F4007259
S31508001D381A611A6942F001021A610160BFF34F8FEE
S31508001D48704700BF003C0240084B1A6922F44072EB
S31508001D581A611A6942F480721A611A6942F0010214
S31508001D681A610180BFF34F8F704700BF003C0240DD
S31508001D78074B1A6922F440721A611A691A611A69B4
S31508001D8842F001021A610170BFF34F8F704700BF16
S31508001D98003C02401A4BDB6813F0020F04D0194ABC
S31508001DA8936943F020039361154BDB6813F0100F12
S31508001DB804D0144A936943F010039361104BDB6807
S31508001DC813F0200F04D00F4A936943F00803936170
S31508001DD80B4BDB6813F0400F04D00A4A936943F0AB
S31508001DE804039361064BDB6813F0800F04D0054A99
S31508001DF8936943F002039361014BF222DA60704754
S31508001E08003C02402C0E0020094B1B69002B01DB05
S31508001E1800207047064B074A5A6002F188325A6012
S31508001E281B69002B01DB002070470120704700BFA3
S31508001E38003C024023016745034A136943F00043FF
S31508001E4813610020704700BF003C024038B50446BD
S31508001E58154B00229A6102F09FFB0546134BDB6877
S31508001E6813F4803F0AD0B4F1FF3FF7D024B102F04B
S31508001E7893FB401BA042F1D903200DE00B4BDB680E
S31508001E8813F0F20F09D1094BDB6813F0010F08D0DC
S31508001E98064B0122DA60002038BDFFF77BFF0120D8
S31508001EA8FAE70020F8E700BF2C0E0020003C0240A5
S31508001EB8F8B51E4C247D012C35D01F4616460D460E
S31508001EC804461A4B01221A754CF25030FFF7BEFF2A
S31508001ED8014698B9032C07D8DFE804F002151A1F3B
S31508001EE8F1B22846FFF744FF4CF25030FFF7AEFF31
S31508001EF801460F4A136923F0010313610B4B0022AD
S31508001F081A750846F8BDB1B22846FFF71DFFEBE774
S31508001F1831462846FFF704FFE6E732463B46284699
S31508001F28FFF7E6FEE0E70221EBE700BF2C0E0020EC
S31508001F38003C0240014B1868704700BF2C0400207B
S31508001F487047002800F0A18038B5044690F820307C
S31508001F58D3B12268136823F00203136002F01CFB4E
S31508001F68054623685A6812F0020F10D002F014FBCF
S31508001F78401B0A28F5D9636A43F4003363620523CC
S31508001F8884F82030012038BDFFF7DAFFE1E71A6840
S31508001F9842F001021A6002F0FFFA054623685A68F9
S31508001FA812F0010F0DD102F0F7FA401B0A28F5D9ED
S31508001FB8636A43F400336362052384F820300120FA
S31508001FC8E1E7227E012A3DD01A6822F080021A60CB
S31508001FD8637E012B3BD02268136823F04003136005
S31508001FE8A37E012B39D02268136823F020031360D7
S31508001FF8E37E012B37D02268136843F01003136079
S31508002008237F012B35D02268136823F00803136051
S31508002018637F012B33D02268136823F00403136007
S31508002028A368E26813432269134362691343626823
S31508002038013A21681343CB6100206062012384F8C2
S315080020482030A0E71A6842F080021A60C0E72268C2
S31508002058136843F040031360C2E72268136843F025
S3150800206820031360C4E72268136823F0100313607B
S31508002078C6E72268136843F008031360C8E72268AE
S31508002088136843F004031360CAE701207047000089
S3150800209890F82030013BDBB2012B05D9436A43F49B
S315080020A8802343620120704770B4434BD3F800225B
S315080020B842F00102C3F80022D3F8002222F47C5227
S315080020C8C3F80022D3F80022486A42EA0022C3F875
S315080020D800224A6902F01F02012000FA02F2D3F828
S315080020E81C42D0430440C3F81C42CB69B3B9324BEF
S315080020F8D3F80C420440C3F80C42CE688D884C6964
S3150800210845EA0645483443F834508E680C884D69C4
S3150800211844EA0644483503EBC5035C60CB69012BE2
S315080021281DD08B69002B32D1234CD4F804320340D6
S31508002138C4F804320B698BBB1F4BD3F814422040F2
S31508002148C3F814020B6A012B2FD01B4AD2F80032A7
S3150800215823F00103C2F80032002070BC7047164B02
S31508002168D3F80C421443C3F80C420E688D884C69A0
S3150800217845EA0645483443F834508E688C894D69D3
S3150800218844EA0644483503EBC5035C60C9E70A4CCC
S31508002198D4F804321343C4F80432CBE70648D0F817
S315080021A814321343C0F81432CCE70349D1F81C3269
S315080021B81A43C1F81C22C8E70064004038B590F8ED
S315080021C82030DBB2012B05D0436A43F4002343626F
S315080021D8012038BD0446022380F8203002681368B7
S315080021E823F00103136002F0D7F9054623685B68F4
S315080021F813F0010F0DD002F0CFF9401B0A28F5D9C4
S31508002208636A43F400336362052384F820300120A7
S31508002218DFE700206062DCE770B490F820400568C4
S31508002228AD68013CE4B2012C65D815F0E05F5CD0D6
S31508002238C5F30165022D05D9436A43F400034362D1
S3150800224801205DE00124AC401C608B68002B39D165
S315080022580E68CB68046843EA465605F118031B015D
S31508002268E65003680C6905F1180603EB06135C606B
S315080022780B7D012B31D0D17993791B0443EA01638D
S31508002288517943EA01231479016823432C0121442F
S31508002298C1F88C31D17893781B0443EA01635178E5
S315080022A843EA0123117802680B432244C2F88831AD
S315080022B8016805F118031B01CA5842F00102CA5001
S315080022C800201DE04C6843EAC403CC68066823432B
S315080022D805F1180424013351C3E7036803EB061311
S315080022E8596841F480715960C5E7436A43F4001395
S315080022F84362012004E0436A43F4802343620120D1
S3150800230870BC704790F82030013BDBB2012B01D92D
S315080023180020704703689B68890631EA030301D0E1
S31508002328012070470020704730B490F82040013CDF
S31508002338E4B2012C00F28A8051B90468E46814F002
S31508002348030F10D1436A43F400134362012082E065
S315080023580468246914F0030F05D1436A43F400138B
S315080023684362012077E0056801F11B0424012C5912
S3150800237804F004049460002C5AD1056801F11B0482
S3150800238824012C59640D1460056801F11B04240105
S315080023982D59C5F34005D560056825446D6805F0CF
S315080023A80F051561056825446D68C5F30725956108
S315080023B805682C446468240C546104680A011444AA
S315080023C8D4F8B8411C7004681444D4F8B841C4F366
S315080023D807245C7004681444D4F8B841C4F3074465
S315080023E89C7004681444D4F8B841240EDC70046858
S315080023F81444D4F8BC411C7104681444D4F8BC418C
S31508002408C4F307245C7104681444D4F8BC41C4F3C3
S3150800241807449C7104682244D2F8BC21120EDA716A
S3150800242871B90268D36843F02003D360002012E02C
S31508002438056801F11B0424012C59E4085460A3E734
S315080024480268136943F020031361EFE7436A43F40C
S3150800245880234362012030BC70470000014B186096
S31508002468704700BF2C04002038B5036813F0010F25
S3150800247875D10D46044603683C4A1A404B68C96834
S315080024880B4329690B43A9690B4313430360AB68DC
S31508002498426822F44052134343606B69826822F407
S315080024A8407213438360324B984216D0314B984298
S315080024B827D0314B984228D0304B984229D0304BF8
S315080024C898422AD02F4B98422CD02F4B98422ED080
S315080024D82E4B984230D0012042E0032000F008F93C
S315080024E800283ED02B68002B3DD0AA69B2F5004FCC
S315080024F827D000EB5300B0FBF3F080B2E060002071
S315080025082EE00C2000F0F4F8EAE7302000F0F0F8A6
S31508002518E6E7C02000F0B6F9E2E74FF4407000F0AD
S31508002528B1F9DDE74FF4406000F0E2F8D8E74FF478
S31508002538405000F0A7F9D3E74FF4404000F0A2F95D
S31508002548CEE75A0802EB4000B0FBF3F04FF6F073FB
S315080025580340C0F342001843E060002000E0012071
S3150800256838BD0120FCE70120FAE700BFF369FFEF51
S31508002578001001400044004000480040004C00405C
S31508002588005000400014014000780040007C0040DC
S315080025981E4A136843F0010313601C4B1B6813F0AB
S315080025A8020FFAD0194A00239360194B136013686F
S315080025B823F0F80343F080031360144B1B6813F0E9
S315080025C8007FFAD1114B1B6813F0006FFAD10F4B35
S315080025D81B6813F0005FFAD10C4B0E4A5A60103A82
S315080025E8C3F88420C3F88820DA6822F4FE42DA6041
S315080025F8DA6842F47F02DA605A6F22F001025A67F3
S315080026085A6F42F080725A670020704700380240B5
S31508002618FFFFF2EA10300024034B9B68C3F3031349
S31508002628024AD35CD840704700380240DC5000089C
S31508002638034B9B68C3F38223024AD35CD84070478E
S3150800264800380240EC500008034B9B68C3F342333A
S31508002658024AD35CD840704700380240EC5000085C
S315080026680D4B5B6803F480039BB90C480A4B5A6800
S3150800267802F03F02B0FBF2F25868C0F3881000FB7C
S3150800268802F05B68C3F3014301335B00B0FBF3F068
S3150800269870470348EAE700BF003802400024F40000
S315080026A800127A0008B5074B9B6803F00C03042B45
S315080026B804D0082B04D1FFF7D3FF02E0024800E054
S315080026C8024808BD0038024000127A000024F400C7
S315080026D810B50446FFF7E6FF2060FFF79DFF606028
S315080026E8FFF7A6FFA0606068FFF7AEFFE06010BDC1
S315080026F808B5032808D00C282DD0B0F5406F51D05E
S31508002708302877D0002008BD584BD3F890300340BE
S3150800271843EA0040564B98420FD0B0F1031F13D036
S31508002728013B984206D0FFF7BDFFFFF775FFFFF795
S315080027388BFFE8E7FFF7B6FFE5E74C4B1B6813F096
S31508002748020F7ED10020DEE7484B1B6F13F0020FFD
S3150800275879D10020D7E7454BD3F89030034043EAB0
S315080027680040444B98420FD0B0F10C1F13D0043BDD
S31508002778984206D0FFF796FFFFF74EFFFFF758FF78
S31508002788C1E7FFF78FFFBEE7384B1B6813F0020F48
S315080027985CD10020B7E7354B1B6F13F0020F57D1F2
S315080027A80020B0E7314BD3F89030034043EA0040A5
S315080027B8314B984210D0B0F10C2F14D0A3F5806392
S315080027C8984206D0FFF76EFFFFF726FFFFF73CFF94
S315080027D899E7FFF767FF96E7244B1B6813F0020F84
S315080027E839D100208FE7214B1B6F13F0020F34D124
S315080027F8002088E71D4BD3F89030034043EA004091
S315080028081E4B98420FD0B0F1301F13D0103B984298
S3150800281806D0FFF747FFFFF7FFFEFFF709FF72E746
S31508002828FFF740FF6FE7114B1B6813F0020F17D12C
S31508002838002068E70D4B1B6F13F0020F12D100201A
S3150800284861E70F485FE74FF400405CE70C485AE732
S315080028584FF4004057E70A4855E74FF4004052E757
S31508002868074850E74FF400404DE700BF00380240DC
S315080028780200030008000C000008000C20003000C5
S315080028880024F40008B5C0280AD0B0F5407F2FD038
S31508002898B0F5405F54D0B0F5404F79D0002008BD58
S315080028A8594BD3F89030034043EA0040574B9842B7
S315080028B80FD0B0F1C01F14D0403B984206D0FFF79E
S315080028C8F1FEFFF7A9FEFFF7B3FEE8E7FFF7EAFE12
S315080028D8E5E74D4B1B6813F0020F40F08180002096
S315080028E8DDE7494B1B6F13F0020F7BD10020D6E7B3
S315080028F8454BD3F89030034043EA0040444B98428E
S3150800290810D0B0F1032F14D0A3F58073984206D0DF
S31508002918FFF7C8FEFFF780FEFFF78AFEBFE7FFF757
S31508002928C1FEBCE7384B1B6813F0020F5DD10020C7
S31508002938B5E7354B1B6F13F0020F58D10020AEE7E9
S31508002948314BD3F89030034043EA0040314B984264
S3150800295810D0B0F1302F14D0A3F58053984206D082
S31508002968FFF7A0FEFFF758FEFFF762FE97E7FFF7A7
S3150800297899FE94E7244B1B6813F0020F3AD10020FE
S315080029888DE7214B1B6F13F0020F35D1002086E720
S315080029981D4BD3F89030034043EA00401E4B98423B
S315080029A810D0B0F1C02F14D0A3F58043984206D0B2
S315080029B8FFF778FEFFF730FEFFF73AFE6FE7FFF7F7
S315080029C871FE6CE7104B1B6813F0020F17D1002035
S315080029D865E70D4B1B6F13F0020F12D100205EE757
S315080029E80E485CE74FF4004059E70C4857E74FF4A0
S315080029F8004054E7094852E74FF400404FE70748B4
S31508002A084DE74FF400404AE7003802408000C0000E
S31508002A180002000300200030008000C00024F400F3
S31508002A280649CB6823F4E0631B041B0C000200F478
S31508002A38E0600343024A1A43CA60704700ED00E0A3
S31508002A480000FA0530B4154BDB68C3F30223C3F15B
S31508002A580704042C28BF04241D1D062D01D9033B91
S31508002A6800E000234FF0FF3505FA04F421EA0401D3
S31508002A78994005FA03F322EA03031943002805DBFC
S31508002A880901C9B2064B195430BC704700F00F004B
S31508002A980901C9B2034B1954F6E700BF00ED00E077
S31508002AA800E400E014ED00E00138B0F1807F0AD2B6
S31508002AB8064B5860064AF02182F8231000209860D1
S31508002AC807221A6070470120704700BF10E000E02F
S31508002AD800ED00E0002301330C4A934211D802693D
S31508002AE8002AF8DA036943F0010303610023013376
S31508002AF8064A934207D8026912F0010FF7D1002057
S31508002B087047032070470320704700BF400D030035
S31508002B1884B010B5044603A880E80E00089B012B6C
S31508002B281DD1A36B23F48033A363E268164B1340C5
S31508002B38E360E36823F44013E3600F9B012B09D095
S31508002B482046FFF7C7FF069B012B14D0BDE81040A7
S31508002B5804B07047E36843F48013E360F0E7E3687A
S31508002B6843F04003E3602046FFF7B4FFA36B43F442
S31508002B788033A363E7E7A36843F00603A360A36863
S31508002B8843F02003A360E1E7BFFFBDFF022A0AD08E
S31508002B980921C26822F47052C260C36843EA8123D5
S31508002BA8C36000207047274B0B44274A934237D9FE
S31508002BB8264B0B44264A934234D9264B0B44264ABD
S31508002BC8934231D9254B0B4402F5C332A0329342BE
S31508002BD82CD9234B0B44234A934229D9224B0B441D
S31508002BE802F5922202F57872934223D91F4B0B44B9
S31508002BF802F5C32202F5207293421DD91C4B0B44D9
S31508002C0802F5B71202F55872934217D9194B0B44B5
S31508002C1802F5122202F5F862934211D80721B8E79D
S31508002C280F21B6E70E21B4E70D21B2E70C21B0E76C
S31508002C380B21AEE70A21ACE70921AAE70821A8E78C
S31508002C480621A6E7405327FFFF340C00401E1BFF4A
S31508002C583F420F0000DC0BFF7F4F1200808CF9FE05
S31508002C6860B6E5FE5FE3160000D3CEFEC05BB3FE92
S31508002C7800CA91FEE05459FE836843F00103836055
S31508002C8800207047836823F001038360002070479B
S31508002C9808B5C36823F0C043C360012909D069B9D8
S31508002CA8C36843F08043C3603220FEF7CDF800209E
S31508002CB808BDC36843F00053C360F5E70120F7E78A
S31508002CC8890141F02001016100230133054A934235
S31508002CD805D8026912F0200FF7D1002070470320A3
S31508002CE8704700BF400D030010230361002301331A
S31508002CF8054A934205D8026912F0100FF7D1002049
S31508002D0870470320704700BF400D0300D0F800380D
S31508002D181943C0F8001800207047000084B0F8B5B9
S31508002D28044607A880E80E00254600230E2B07D878
S31508002D3803F1400204EB8202002151600133F5E7F2
S31508002D48119B03BBA36B23F40013A363236843F007
S31508002D5840032360236843F0800323600023C4F8F4
S31508002D68003E04F50066D4F80038C4F800380C9B11
S31508002D78012B0DD0032B1CD1099BABB9002120468A
S31508002D88FFF7C4FF19E0A36B43F40013A363E5E751
S31508002D98099B23B900212046FFF7B8FF0DE001215A
S31508002DA82046FFF7B3FF08E001212046FFF7AEFFEC
S31508002DB803E003212046FFF7A9FF10212046FFF765
S31508002DC87FFF074600B101272046FFF78DFF00B1B0
S31508002DD80127002333617361F3610AE0C3B94FF031
S31508002DE80060C2F8000900220A614FF67F328A603D
S31508002DF80133079A9A4210D905EB431202F5106176
S31508002E08D2F800090028E9DB0020C2F80009EAE739
S31508002E184FF09040C2F80009E5E700230AE0C3B975
S31508002E284FF00060C2F8000B00220A614FF67F32A5
S31508002E388A600133079A9A4210D905EB431202F5BC
S31508002E483061D2F8000B0028E9DB0020C2F8000B35
S31508002E58EAE74FF09040C2F8000BE5E7336923F438
S31508002E68807333610A9B012B1BD00022A2616FF085
S31508002E78804262611BB9A36943F01003A361A26982
S31508002E880E4B1343A3610D9B1BB1A36943F00803BB
S31508002E98A361119B012B0BD03846BDE8F84004B056
S31508002EA87047074A3263316B064A0A433263DCE7DE
S31508002EB8A269054B1343A361EEE700BF00383C80BF
S31508002EC8000180000300010004000040D0F808381B
S31508002ED813F0060307D0062B18BF022B01D00020D3
S31508002EE870470220704700207047000070B40B78BE
S31508002EF84A78012A20D0D0F81C2803F00F060124A6
S31508002F08B44042EA0442C0F81C2800EB4310D0F843
S31508002F18003B13F4004F0CD1D0F8002B8B68C3F391
S31508002F280A03C97843EA81431343134A1A43C0F884
S31508002F38002B002070BC7047D0F81C4803F00F0619
S31508002F48B24092B22243C0F81C2800EB4310D0F8CE
S31508002F58002912F4004FECD1D0F800498A68C2F368
S31508002F680A02C97842EA814242EA8353234302495C
S31508002F781943C0F80019DCE70080001070B40B7814
S31508002F884A78012A1FD0D0F83C5803F00F060124C6
S31508002F9804FA06F625EA0645C0F83C58D0F81C583F
S31508002FA8097801F00F018C4025EA0444C0F81C484A
S31508002FB800EB4310D0F8002B124B1340C0F8003B27
S31508002FC8002070BC7047D0F83C6803F00F0402FA7A
S31508002FD804F4A4B226EA0404C0F83C48D0F81C480D
S31508002FE8097801F00F018A4092B224EA0202C0F871
S31508002FF81C2800EB4310D0F80039034A1A40C0F8D9
S315080030080029DDE70078F3EF007833EC70B40B7825
S315080030184C78012C24D000EB431000F530631D6969
S315080030283A4C2C401C611D69394C2C401C614C6972
S315080030380CB18C684C611C6944F400241C611C6939
S315080030488D68C5F312052C431C61012A59D0D0F89E
S31508003058003B43F00443C0F8003B002070BC7047AF
S315080030684C6954BB00EB4314D4F81069284D354015
S31508003078C4F81059D4F8105945F40025C4F810595D
S31508003088D4F81069214D3540C4F81059012A30D0B2
S315080030984A694AB1D0F83428097801F00F040121A1
S315080030A8A1400A43C0F8342800EB4310D0F8002999
S315080030B842F00442C0F80029CFE700EB431404F5B0
S315080030C810642669114D354025612669104D35402D
S315080030D825614E698D68AE4200D94D61256945F46A
S315080030E80025256125694E69C6F31206354325610B
S315080030F8CCE70A69002AD7D000EB4311C1F814298E
S31508003108D2E7CA68002AA2D05A61A0E70000F8FFE9
S31508003118FFFF07E070B49DF80C4064B903339E08B6
S31508003128B44208D200EB023303F5805351F8045B26
S315080031381D600134F4E7002070BC7047F0B583B011
S315080031480B784C78012C29D000EB431303F530642F
S315080031582669704D3540256126696F4D35402561CC
S315080031684D69002D40F0A88025698E68C6F31206B9
S3150800317835432561256945F400252561012A00F0AE
S31508003188B080CA78012A00F0B280D3F8002B42F042
S315080031980442C3F8002B002003B0F0BD4C69002C8C
S315080031A839D100EB4314D4F810695B4D3540C4F89F
S315080031B81059D4F8105945F40025C4F81059D4F80C
S315080031C81069544D3540C4F81059012A55D0CC78A1
S315080031D8012C0BD04C694CB1D0F834480D7805F061
S315080031E80F060125B5402C43C0F83448CC78012C85
S315080031F84BD000EB4313D3F8004944F00444C3F812
S315080032080049CB78012BC6D100928B8A0A78C968FF
S31508003218FFF780FFBFE700EB4314D4F810693D4D6C
S315080032283540C4F81059D4F810693B4D3540C4F8F0
S315080032381059D4F810694D698F683D44013DB5FBAE
S31508003248F7F5364F07EAC5453543C4F81059D4F893
S3150800325810594E69C6F312063543C4F8105904F5D1
S315080032681064CD78012DB0D1256925F0C0452561B2
S31508003278256945F000552561A7E70C69002CB5D0E6
S3150800328800EB4315C5F81449B0E7D0F8084814F414
S31508003298807F08D100EB4315D5F8004944F000545F
S315080032A8C5F80049A5E700EB4315D5F8004944F0E9
S315080032B88054C5F800499CE78E683544013DB5FB3E
S315080032C8F6F52669154F07EAC5473E432661276975
S315080032D88E68ADB206FB05F5C5F312053D432561B3
S315080032E84CE7CA68002A3FF44CAF626149E7D0F850
S315080032F8082812F4807F06D1D3F8002B42F0005232
S31508003308C3F8002B41E7D3F8002B42F08052C3F8E4
S31508003318002B3AE70000F8FFFFFF07E00000F81F58
S3150800332803329208002393420CD210B400F5805455
S31508003338246841F8044B01339342F7D308465DF8ED
S31508003348044B7047084670470B784A78012A14D008
S3150800335800EB4310D0F8002B002A06DB2BB1D0F877
S31508003368003B23F08043C0F8003BD0F8003B43F409
S315080033780013C0F8003B0020704700EB4310D0F854
S315080033880029002A06DB2BB1D0F8003923F0804340
S31508003398C0F80039D0F8003943F40013C0F80039EA
S315080033A8E9E70B784A78012A0ED000EB4310D0F8E3
S315080033B8003B23F40013C0F8003BCB78023BDBB292
S315080033C8012B15D90020704700EB4310D0F80039B7
S315080033D823F40013C0F80039CB78023BDBB2012B83
S315080033E8F0D8D0F8003943F08053C0F80039E9E737
S315080033F8D0F8003B43F08053C0F8003BE2E738B505
S315080034080546044600220E2A09D804EB42134FF64D
S315080034187F31C3F80819C3F8081B0132F3E70022FD
S31508003428C5F81028C5F81428C5F81C282846FFF733
S315080034385BFC034608B1184638BD10212846FFF735
S315080034483FFC0346F7E7D0F8003823F4FE63C0F8D4
S315080034580038D0F80038090101F4FE610B43C0F8BA
S3150800346800380020704708B5D0F8043823F002035E
S31508003478C0F804380320FDF7E7FC002008BD08B5A6
S31508003488D0F8043843F00203C0F804380320FDF7DF
S31508003498DBFC002008BD4269806910407047D0F8F7
S315080034A8183800F50060C0691840000C7047D0F855
S315080034B8183800F50060C069184080B2704700EBFC
S315080034C84111D1F8082B00F5006040691040704793
S315080034D810B4D0F81048D0F8343801F00F02D340A9
S315080034E8DB01DBB2234300EB411000F5106080686E
S315080034F818405DF8044B7047406900F001007047B2
S31508003508D0F800290B4B1340C0F8003900F50063C2
S315080035189A6802F00602042A05D05A6842F48072AC
S315080035285A6000207047D0F8002942F00302C0F814
S315080035380029F2E700F8FFFF10B4046C154B9C420B
S3150800354803D9D0F8003B002B16DB0024C0F8104B33
S31508003558D0F8104B44F40024C0F8104BD0F8104BA0
S3150800356844F01804C0F8104BD0F8104B44F0C04487
S31508003578C0F8104B012903D000205DF8044B7047AA
S31508003588C0F8142BD0F8003B43F08023C0F8003B62
S31508003598F2E700BF0A30544F084B1A6922F4407202
S315080035A81A611A6942F004021A611A6942EA002085
S315080035B840F480301861BFF34F8F7047003C0240D3
S315080035C810B449B1012923D0022902D04FF4407218
S315080035D803E04FF4007200E000220F4B1C6924F444
S315080035E840741C61196911431961196921F0F801B8
S315080035F819611A6942EAC00242F002021A611A6996
S3150800360842F480321A61BFF34F8F5DF8044B704756
S315080036184FF48072E1E700BF003C0240214B1B7D56
S31508003628012B3CD070B50E4604461E4B01221A756E
S315080036384CF25030FEF70AFC014658BB4FF0FF33F0
S3150800364833602368012B16D06568A368626813443B
S31508003658AB421FD9217B2846FFF7B2FF4CF2503000
S31508003668FEF7F4FB104A136923F07A03136101463F
S3150800367878B90135E9E7207BFFF78EFF4CF2503021
S31508003688FEF7E4FB0146084A136923F004031361AD
S3150800369800E03560034B00221A75084670BD022102
S315080036A8084670472C0E0020003C024030B40468D7
S315080036B8606A29B940EA0240A062002030BC704717
S315080036C80D46A36A00EB13400023691E8B4209D2F4
S315080036D803F1400104EB8101496800EB114001330D
S315080036E8DBB2F2E740EA024005F13F0104EB81014B
S315080036F84860E2E703685962002070470246036893
S315080037080121C0F8FC13002082F8F4039A6942F0F4
S3150800371800629A61596D024A0A435A65704700BFA2
S31508003728030000107047000012230B8000487047FA
S315080037385404002004230B800048704768040020BE
S315080037480023934216D230B40BE0373401F81340FD
S3150800375800015C00013400250D550133DBB29342A4
S3150800376806D2040F092CF0D8303401F81340EFE7D5
S3150800377830BC70477047000038B50A4B18680433E0
S315080037881C6804331B68C01800D138BD064D0822CA
S31508003798A91CFFF7D5FF042205F112012046FFF7F9
S315080037A8CFFFF2E720F4F01F6C04002008B51A23AF
S315080037B80B80FFF7E1FF014808BD00BF6C04002035
S315080037C808B50A4628B905490548FDF72CF90348F6
S315080037D808BD02490248FDF726F9F8E7480E002011
S315080037E82451000810B5044C0A4621460348FDF73B
S315080037F81AF9204610BD00BF480E002014510008CB
S3150800380808B50A4628B905490548FDF70CF90348D5
S3150800381808BD02490248FDF706F9F8E7480E0020F0
S31508003828F450000808B50A4628B905490548FDF7B9
S31508003838FAF8034808BD02490248FDF7F4F8F8E71C
S31508003848480E0020FC500008014B1880704700BF3E
S315080038580A05002008B500F097FE0E4B1B6898422B
S315080038680FD30D4B1B786BB90B4B01221A700B4BF8
S3150800387880229A6100F088FE094B1B881844054B7C
S31508003888186008BD044B00221A70044B4FF4000256
S315080038989A61EFE7100500200C0500200004024095
S315080038A80A050020024B4FF400029A61704700BFD0
S315080038B80004024008B5054B1B6913F4005F01D0E4
S315080038C8002008BDFFF7EEFF0120FAE700080240CE
S315080038D808B56420FFF7B8FF08BD08B5FFF7BAFFB3
S315080038E808BD70477047704708B5304A136823F013
S315080038F80F0343F007031360136803F00F03072B3E
S315080039084ED12B4B1A6842F440421A601A6842F4A0
S3150800391880321A6003F5E4331A6842F480221A6082
S315080039281A6842F480321A60224B1B6813F4003F67
S31508003938FAD0204B5A6820491140204A0A435A604F
S315080039485A681F4911401F4A0A435A601A6842F0C2
S3150800395880721A60174B1B6813F0007FFAD0154B54
S315080039689A6822F0F0029A609A6822F4E05242F4C1
S31508003978A0529A609A6822F4604242F400429A6019
S315080039889A6822F0030242F002029A60094B9B6881
S3150800399803F00C03082BF9D10B48FEF75FFD08BDA9
S315080039A86A210A4800F0C0FAABE700BF003C0240AB
S315080039B800700040003802400080BCFF086C4000D8
S315080039C80080BFF0086C400900E6DF0C3851000893
S315080039D808B5FDF72DFAFFF787FF08BD08B5FFF705
S315080039E8F7FF00F0ADFA00F0B9FAFCE72DE9F04365
S315080039F891B04C4C636C43F480436364636C03F482
S31508003A0880430993099B236C43F080532364236CF2
S31508003A1803F080530893089B236B43F00103236341
S31508003A28236B03F001030793079B236B43F00203F9
S31508003A382363236B03F002030693069B236B43F069
S31508003A4804032363236B03F004030593059B236B85
S31508003A5843F008032363236B03F008030493049BCA
S31508003A68236C43F480232364236C03F48023039391
S31508003A78039B236C43F000732364236C03F00073E1
S31508003A880293029B80230A9301230B9300250C9526
S31508003A980D950E95DFF89C800AA94046FEF78EF824
S31508003AA84FF40003C8F818304FF400530A930B95DF
S31508003AB80E950AA91C48FEF781F84FF44079CDF807
S31508003AC8289002270B9703260C960D950E95072323
S31508003AD80F930AA91548FEF771F8CDF828900B97A1
S31508003AE80C960D950E9509230F930AA94046FEF7DD
S31508003AF865F84FF4C0530A930B970C960D950E95D7
S31508003B080A230F930AA90A48FEF758F8636B43F085
S31508003B1880036363636B03F080030193019B11B011
S31508003B28BDE8F0830038024000080240000C024055
S31508003B38000002400004024010B5FEF729FD1B4CA0
S31508003B484FF40003A3611A48FDF77AFF1948FDF7F1
S31508003B5877FF2046FDF774FF1748FDF771FF174BE7
S31508003B685A6B22F080025A631A6C22F000721A64A1
S31508003B781A6C22F480221A641A6B22F008021A6355
S31508003B881A6B22F004021A631A6B22F002021A63ED
S31508003B981A6B22F001021A631A6C22F080521A6410
S31508003BA85A6C22F480425A6410BD00BF00040240D1
S31508003BB8000C02400008024000000240003802409B
S31508003BC82023038000487047C00400200A23038086
S31508003BD800487047E004002008B590F87432032BB3
S31508003BE801D0002008BD01F0E3F9FAE708B501F0AD
S31508003BF8DFF9002008BD08B5084601F00DFA0020CF
S31508003C0808BD000008B50B7813F0600F06D14B788D
S31508003C180A2B14D00B2B17D0062B01D0002008BD71
S31508003C284B881B0A212B04D00B491722FCF7A7FB44
S31508003C38F4E7CA88172A28BF17220849F6E701228F
S31508003C480749FCF79CFBE9E78B7813B9044A136024
S31508003C58E4E7FCF7EEFBE1E7C9040020D2040020FC
S31508003C681405002010B50446812100F02DF901211C
S31508003C78204600F029F9002010BD000010B50446BA
S31508003C8840230222812100F014F94023022201214F
S31508003C98204600F00EF94023034A0121204600F089
S31508003CA83BF9002010BD00BF4810002000487047A7
S31508003CB84810002008B500F57171D0F80004FCF723
S31508003CC816FF08BD08B5C1EBC10293000344D3F833
S31508003CD80822D0F80004FCF738FF08BD08B5C1EB80
S31508003CE8C102930003449A6CD0F80004FCF777FFE6
S31508003CF808BD08B5D0F80004FDF717F808BD000098
S31508003D0810B50446C3684BB1022B01D1012106E060
S31508003D189121074800F008F9012100E00021D4F8AC
S31508003D280004FCF7F0FFD4F80004FCF7C4FF10BD44
S31508003D384051000810B50446D0F80004FCF7E6FF21
S31508003D482268D2F8003E43F00103C2F8003E236A0F
S31508003D5823B1044A136943F006031361FFF7C2FD4A
S31508003D6810BD00BF00ED00E010B50446FFF7BBFD27
S31508003D78D4F80004FCF7D3FF10BD08B5D0F8000442
S31508003D88FCF7E3FF08BD08B5D0F80004FCF7DBFF2D
S31508003D9808BD10B504460120FFF7A3FDD4F80004B2
S31508003DA8FCF7D5FF10BD10B504460020FFF799FDAE
S31508003DB8D4F80004FCF7CDFF10BD000003780BB15A
S31508003DC80020704710B503461748C0F80034C3F8F2
S31508003DD898024FF0A0430360062343600222C2609C
S31508003DE80023036182610122C26103624362C362DE
S31508003DF80363FDF7A7F880B90B4C80212046FFF727
S31508003E0879FC402200212046FFF750FC8022012138
S31508003E182046FFF74BFC002010BD40F22511034849
S31508003E2800F082F8E8E700BF881000204051000833
S31508003E38D0F8983211F0800F08D101F07F01C1EB54
S31508003E48C1018A00134493F8FE01704701F07F0107
S31508003E58C1EBC1018A00134493F83E00704708B5C0
S31508003E68D0F89802FDF741FD08BD022807D8DFE813
S31508003E7800F002060400002070470120704702205F
S31508003E88704708B5D0F89802FDF723F9FFF7EDFF54
S31508003E9808BD08B5D0F89802FDF7E6F8FFF7E5FF7C
S31508003EA808BD08B5D0F89802FDF7F3F8FFF7DDFF67
S31508003EB808BD10B51C4613462246D0F89802FDF7E9
S31508003EC870FCFFF7D2FF10BD08B5D0F89802FDF7C9
S31508003ED8A8FCFFF7CAFF08BD08B5D0F89802FDF791
S31508003EE837FDFFF7C2FF08BD08B5D0F89802FDF7F9
S31508003EF870FDFFF7BAFF08BD08B5D0F89802FDF7B8
S31508003F083CFCFFF7B2FF08BD08B5D0F89802FDF7E4
S31508003F18F5FCFFF7AAFF08BD08B5D0F89802FDF723
S31508003F28B6FCFFF7A2FF08BD08B500F005F8FCE7E0
S31508003F3808B5FFF7CDFC08BD08B5FFF7CEFC08BDE8
S31508003F4808B500F07BFEFFF7F3FF00F0FBFA01F077
S31508003F588FF800F057F800F049F808BD08B5FFF7DC
S31508003F68EBFF00F003FB00F061F800F001F808BD6C
S31508003F7808B500F0DFF8012803D00B4B1B78012B96
S31508003F8800D008BD00F000FB084B1B68084A1268F9
S31508003F98134403F5FA739842F3D3034B00221A70B5
S31508003FA800F050FEEDE700BF1C05002018050020AC
S31508003FB820050020014B1860704700BF180500202F
S31508003FC8014B1868704700BF1805002008B5054B4F
S31508003FD81B78012B00D008BD00F0D6FA024B1860F2
S31508003FE8F9E700BF1C0500202005002008B5044B8A
S31508003FF801221A70FFF7EAFFFFF7BAFF08BD00BFEC
S315080040081C05002010B500F005FA00F0B7FB064CB1
S315080040180123237000F0EAFA0023237000F0FEFE5D
S315080040280223237010BD00BFEA04002000B583B040
S315080040380DF10701184800F01DFC012810D00DF1F4
S315080040480701154800F008FB012812D00DF10701F1
S31508004058114800F061FF012814D003B05DF804FB8D
S315080040680E4B01221A709DF807100B4800F0F2F95A
S31508004078E5E70A4B00221A709DF80710064800F073
S31508004088E9F9E3E7054B02221A709DF8071002487A
S3150800409800F0E0F9E1E700BF24050020EA04002063
S315080040A808B500F0FFFE08BD38B504460D460E4BA8
S315080040B81B78012B09D00C4B1B7853B10A4B1B787C
S315080040C8022B0BD000F0BEF938BDC9B200F0ACFB24
S315080040D8F1E7E9B2204600F0A3FAEFE7E9B220468D
S315080040E800F0F0FEEEE700BFEA040020074B1B7855
S315080040F8022B05D0032B05D0012B05D0402070478D
S315080041083F2070470020704708207047EA040020BF
S31508004118074B1B78022B05D0032B05D0012B05D09E
S31508004128402070473F207047002070470820704796
S31508004138EA04002008B500F07BF9034600B101231C
S31508004148184608BD014B00225A70704764050020BE
S31508004158034BFE22DA7018710222A3F8442070472E
S315080041686405002010B5054C00232370FFF7EAFF05
S31508004178FF23E3700123A4F8443010BD640500202A
S31508004188064BFF22DA7000221A71597859719A710A
S31508004198DA711A720622A3F84420704764050020CB
S315080041A808B50020FFF7D4FF08BD0000074BFF221B
S315080041B8DA70074A9A6400221A715A719A710722A4
S315080041C8C3F807200822A3F844207047640500208E
S315080041D84C510008044BFF22DA7042689A6401229F
S315080041E8A3F84420704700BF6405002008B53120AD
S315080041F8FFF7AEFF08BD000038B5084CFF23E3708B
S31508004208002525716571FFF771FFA071E5712572A3
S3150800421865720723A4F8443038BD00BF640500203A
S3150800422838B5FFF78FFF0E4C01252570FF23E3707D
S315080042381023237100236371FFF758FFA071FFF756
S3150800424867FFE071FFF764FFC0F307202072657205
S31508004258A5720823A4F8443000F00AFF38BD00BF49
S315080042686405002038B50546FFF740FF6A7890428E
S315080042780FD90A4CA16C201D00F004FDFF23E3703A
S315080042886A78A36C1344A3646B780133A4F84430A2
S3150800429838BD2220FFF75CFFFAE700BF6405002057
S315080042A838B50446FFF722FF6378984211D9616842
S315080042B80A4DA9646278281D00F0E4FCFF23EB7018
S315080042C86278AB6C1344AB6463780133A5F8443061
S315080042D838BD2220FFF73CFFFAE700BF6405002037
S315080042E8F8B50546174600244E1E39B115F8013BA0
S315080042F81C44E4B2FFF720FE3146F5E73C6001208E
S31508004308F8BD000010B5084CFF23E370E21D4168AC
S31508004318A06CFFF7E5FF207100236371A3710823DA
S31508004328A4F8443010BD00BF6405002038B505461A
S315080043380D4B9C6CFFF7DAFE6A1C411E204600F0FE
S315080043489BFE60B1084CFF23E370FFF7CFFE0138E8
S31508004358A36C0344A3640123A4F8443038BD312070
S31508004368FFF7F6FEFAE700BF6405002010B5044615
S31508004378FFF7BCFE01386378984213DD114BFF221C
S31508004388DA700122A3F84420617879B1A21C0D4B92
S31508004398986C00F071FE88B161780A4A936C0B44F0
S315080043A8936410BD2220FFF7D3FEFAE700F074FEE7
S315080043B80028F6D13120FFF7CBFEF2E73120FFF7C8
S315080043C8C7FEEEE76405002008B54168074B986CF8
S315080043D800F056FE30B1054BFF22DA700122A3F829
S315080043E8442008BD3120FFF7B3FEFAE7640500202C
S315080043F808B500F027FC034BFF22DA700122A3F860
S31508004408442008BD6405002008B589B2FFF74CFEAC
S3150800441808BD0000054B00221A709A6483F84320E9
S31508004428A3F844209A705A70704700BF64050020A4
S31508004438034B1B780BB1012070470020704700BF5B
S3150800444864050020024B002283F84320704700BF0A
S315080044586405002008B50378FF2B23D0354A12785F
S31508004468012A2BD1C93B352B53D8DFE803F0405234
S31508004478524F52524C434946525252525252525233
S3150800448852525252525252525252525252525252F6
S315080044985252525252525252312B282E525252349A
S315080044A852373A3DFFF7BCFE224B93F84330012BAF
S315080044B833D0204BB3F94410002932DC08BDFFF786
S315080044C8D1FEF1E7FFF7ECFEEEE7FFF783FEEBE731
S315080044D8FFF718FFE8E7FFF769FEE5E7FFF760FE6D
S315080044E8E2E7FFF74DFEDFE7FFF73CFEDCE7FFF7FD
S315080044F81DFFD9E7FFF73AFFD6E7FFF77DFED3E7B3
S31508004508FFF762FFD0E7FFF773FFCDE7FFF76EFE09
S31508004518CAE72020FFF71CFEC6E71020FFF718FE9B
S31508004528C7E71846012380F843300330FFF76CFFC6
S31508004538C4E700BF64050020014B00221A607047D3
S3150800454810E000E008B5FFF7F7FF054B054A5A6083
S3150800455800229A6005211960034B1A6008BD00BF3E
S3150800456810E000E0BF4B0300B0050020044B1B68B1
S3150800457813F4803F03D0034A136801331360704766
S3150800458810E000E0B005002008B5FFF7EFFF014B83
S31508004598186808BDB005002008B5FFF7F5FF08BD7F
S315080045A870470000054BDB6913F0200F04D0034B56
S315080045B85B6A037001207047002070470048004076
S315080045C810B5094B9862FFF7DFFF00F10A04064B9E
S315080045D8DB6913F0800F05D1FFF7AEFCFFF7D4FFB0
S315080045E8A042F4D910BD00BF0048004010B588B0F5
S315080045F84FF46143019300230293039304930C2217
S31508004608059206930793054C01A92046FDF72CFF4A
S31508004618236843F00103236008B010BD0048004032
S3150800462870B506460D4640290ED82846FFF7C8FF36
S315080046380024ABB2A3420CD9FFF77EFC305DFFF726
S31508004648BFFF0134A4B2F4E781210248FFF76CFCE6
S31508004658EBE770BD5451000870B5254B1C78BCB9FA
S315080046682448FFF79FFF012801D0204670BD214B3B
S315080046781B78013BDBB23F2BF7D8FFF785FF1E4BAC
S3150800468818601E4B00221A70194B01221A70ECE7A3
S3150800469806460D46194B1B78013316481844FFF78A
S315080046A881FF0446012815D1144B1A780132D2B273
S315080046B81A70104B1B789A4201D00024D5E7104986
S315080046C8304600F0DFFA0A4B00221A700B4B1B78AB
S315080046D82B70CAE7FFF758FF074B1B6864339842E5
S315080046E803D90024024B1C70BFE70024BDE700BFAE
S315080046F8F5050020B4050020F8050020F605002079
S31508004708B50500202DE9F04184B004460D46174644
S3150800471898466846FDF7DCFF0299164BA3FB01315C
S315080047288909002201E00132D2B2112A1DD8124B9A
S3150800473813F8120003EB420393F801C000EB0C03CD
S3150800474803FB0443B1FBF3FE03FB1E16002EEAD156
S315080047581FFA8EF32B80013B9BB2B3F5806FE2D22A
S31508004768387088F800C0012000E0002004B0BDE8D1
S31508004778F08100BFD34D6210A451000870B58CB003
S315080047880023ADF82E308DF82D308DF82C300BAB74
S315080047980DF12D020DF12E014FF4FA70FFF7B2FF55
S315080047A8002835D01D4C1E4B2360002525766576D6
S315080047B8A5760126E67625776577A560E5609DF8EE
S315080047C82D30013B1B0423619DF82C30013B1B054A
S315080047D86361BDF82E3063602046FDF7B2FB069587
S315080047E8079508964CF6E043019302954FF6E07351
S315080047F8039304230493059509960E230A9301A99E
S315080048082046FDF745FC2046FDF7D8FC0CB070BDE0
S31508004818B5210448FFF788FBC4E700BFFC0500205C
S31508004828006400407C51000810B588B040F2E17376
S315080048380293002304930593069101AB024602A945
S315080048480B48FDF7E9FC08B108B010BDFFF79CFE58
S3150800485800F1320401990648FDF754FD0028F3D003
S31508004868FFF76AFBFFF790FEA042F3D9ECE700BF13
S31508004878FC05002010B588B00C46034601AA00219D
S315080048880A48FDF751FD60B9019A40F267639A42F2
S3150800489801D0002006E0039B33B9059B237001204D
S315080048A800E0002008B010BD0020FBE7FC0500204A
S315080048B838B50546002401E00134E4B2062C15D8BB
S315080048C8FFF73AFB04EB44029300094AD358AB4274
S315080048D8F2D804EB44029100054A0A445268134484
S315080048E8AB42E9D9024B0B44187A00E0FF2038BDE1
S315080048F8C851000808B5C1F3080353B903688B42C1
S3150800490809D040F8041B4FF4007200F0BBF90120E7
S3150800491808BD0020FCE70120FAE72DE9F041074623
S31508004928FDF772FA002400E001347F2C14D83E689B
S31508004938A30006EB03083B445D68FFF7FDFA2A4621
S31508004948002341460220FDF7B3FA38B956F8243051
S31508004958AB42E9D0002402E0012400E00024FDF778
S315080049686BFA2046BDE8F08138B50D460C4B9842DF
S3150800497811D004460B4B994207D1094C29462046C3
S31508004988FFF7B8FF48B1204638BDFFF7C6FF00282D
S31508004998F4D10024F7E7044CF0E70024F3E700BF56
S315080049A82808002000800008240600202DE9F04188
S315080049B806460C4617461D46DFF8748001EA0808BD
S315080049C80368B3F1FF3F07D0336843450BD1336813
S315080049D8E41A3444043415E04146FFF78BFF0346CE
S315080049E80028F1D11FE041463046FFF7BDFF0646CD
S315080049F80028ECD1002316E017F8013B04F8013B20
S31508004A08013D0FD0FFF798FA331DE31AB3F5007F77
S31508004A18F2D308F500713046FFF7A6FF064628B117
S31508004A28041DE9E701231846BDE8F0810023FAE7E3
S31508004A3800FEFFFF70B586B004460E4600230193B4
S31508004A48884219D80125ECB1072E1FD8DDB10023F5
S31508004A5802930223059301230493FDF7D5F9B4427B
S31508004A680DD8FFF769FA039401A902A8FEF7D6FD3F
S31508004A7820B90134E4B2F2E70025E4E70025FDF79A
S31508004A88DBF900E00025284606B070BD0025FAE7E0
S31508004A984FF0FF33024A1360024A1360704700BF9B
S31508004AA8240600202808002070B54B1E134C241A2B
S31508004AB8A34201D9002070BD16460D460446FFF7E5
S31508004AC8F7FEFF2811D028190138FFF7F1FEFF284D
S31508004AD80BD00B4B23400B4A934208D02B46324641
S31508004AE821460948FFF762FFE5E70020E3E72B467A
S31508004AF8324621460548FFF759FFDCE7FFFF0F084E
S31508004B0800FEFFFF00800008240600202808002071
S31508004B184A1E0D4B1B1A9A4201D90020704770B5D8
S31508004B280C460546FFF7C4FE064660190138FFF726
S31508004B38BFFEFF2818BFFF2E01D1002070BD014611
S31508004B483046FFF777FFF9E7FFFF0F08104B1B689A
S31508004B58B3F1FF3F19D000B583B00D4A5368916881
S31508004B680B44D1680B4411690B4451690B4491698C
S31508004B780B44D26913445B42019301AA04210548F0
S31508004B88FFF792FF03B05DF804FB0120704700BFEA
S31508004B9828080020C88100080D4B1B680D4A1268B2
S31508004BA81A440D4B1B6813440C4A126813440C4AE2
S31508004BB812681A440B4B1B681A440B4B1B681344A0
S31508004BC80A4A1268DA4201D0002070470120704765
S31508004BD80080000804800008088000080C80000887
S31508004BE8108000081480000818800008C88100088A
S31508004BF808B50E4B1B68B3F1FF3F07D10C4B1B6872
S31508004C08B3F1FF3F09D10123184608BD0748FFF746
S31508004C1884FE03460028F1D1F6E70548FFF77DFE2E
S31508004C2803460028F0D00123EEE700BF2808002035
S31508004C3824060020004870470080000808B500F0E0
S31508004C4836FA08BD10B500F01FFA00B910BDFEF710
S31508004C5831FE0028FAD0FFF723FAFFF76DFCFCF7B8
S31508004C68ABF800F015FA054B0340054A936000F0C7
S31508004C780FFA446800F01DFAA047E7E780FFFF1F10
S31508004C8800ED00E070B50D460446531E9EB23AB1D3
S31508004C9815F8013B04F8013BFFF74EF93246F4E7ED
S31508004CA870BD0000094B03F11801002232B19A744D
S31508004CB800225A61064B054A1A6070479A74596168
S31508004CC8183318310132D2B2F0E700BF6C0A002057
S31508004CD89C0A00200A4B1B6883B110B45C69084A11
S31508004CE8146019749860D86000225A7418600139DB
S31508004CF808445860987C5DF8044B7047FF20704755
S31508004D089C0A002038B504460D4601281CD86200BE
S31508004D182244D100114B0B445A7C1B7C9A4219D069
S31508004D280E4B0B44DA6815705A7C01325A74DA68E5
S31508004D380132DA605B689A420ED9084A0846515821
S31508004D480244D160012038BD4FF4E0710448FFF7EA
S31508004D58EBF8DCE70020F6E70120F4E76C0A002008
S31508004D681C52000808B50146024B1878FFF7CAFF17
S31508004D7808BD00BFA00A002038B504460D4601281C
S31508004D881ED804EB4403DA00124B13445B7CEBB1E0
S31508004D9862002244D1000F4B0B449A6812782A7095
S31508004DA85A7C013A5A749A6801329A605B689A4240
S31508004DB80ED9084A0846515802449160012006E06F
S31508004DC84FF4F1710448FFF7AFF8DAE7002038BD69
S31508004DD80120FCE76C0A00201C52000808B50146A9
S31508004DE8024B1878FFF7C8FF08BD00BFE40A002081
S31508004DF810B50446012806D804EB4404E200054B1E
S31508004E081344587C10BD40F202210348FFF78CF87A
S31508004E18F2E700BF6C0A00201C52000838B5FFF7F5
S31508004E2841FF1A4C4021601CFFF754FF2070184DAB
S31508004E384021681CFFF74EFF28702378FF2B1BD0EC
S31508004E48FF2819D0134C002213492046FBF706FE03
S31508004E5812492046FBF72BFE0120FEF742FD2046A5
S31508004E68FBF72CFED4F89802FCF763FCFFF7A8F8C2
S31508004E78B0F5FA6F05D338BD85210948FFF754F808
S31508004E88E0E74FF4FA60FFF795F8F4E7A00A002080
S31508004E98E40A0020280B0020380400208804002093
S31508004EA81C52000810B5064CD4F89802FCF753FCB7
S31508004EB82046FBF7EAFD0020FEF713FD10BD00BFEC
S31508004EC8280B002070B506460D463F2906D8284601
S31508004ED8FFF748FF012806D100240FE0B9210D483D
S31508004EE8FFF722F8F3E7BD210A48FFF71DF8F3E7AD
S31508004EF8C6210848FFF718F80134A4B2ABB2A34292
S31508004F0807D9FFF719F8305DFFF72CFF0128F3D00A
S31508004F18EEE770BD1C52000870B506460D461F4BD5
S31508004F28D3F89802FCF798F91D4B1C789CB91D48CC
S31508004F38FFF754FF012801D0204670BD194B1B788E
S31508004F48013BDBB23E2BF7D8154B01221A70164BDC
S31508004F5800221A70F0E7144B1B78013311481844DD
S31508004F68FFF73CFF0446012801D00024E4E70E4B6E
S31508004F781A780132D2B21A700A4B1B789A4201D0B3
S31508004F880024D9E709493046FFF77CFE044B00227E
S31508004F981A70054B1B782B70CEE700BF280B00202C
S31508004FA8040E0020C40D0020050E0020C50D0020A3
S31508004FB830B583B0144B1878FFF71AFF08B30546BF
S31508004FC8402800D9402500240AE04FF4A3710F4869
S31508004FD8FEF7AAFF9DF807200D4B1A550134E4B2CF
S31508004FE8A54208D90DF10701074B1878FFF7C4FE43
S31508004FF80128EFD0E9E7ABB2054A81210548FEF753
S3150800500883FF03B030BD00BFA00A00201C52000869
S315080050182C0A0020280B002070B50446FEF746FE29
S31508005028064621460F48FEF71AFF85B2002406E011
S315080050384FF4B4710C48FEF777FF0134A4B2AC42BA
S3150800504807D2315D094B1878FFF75CFE0128F4D0C2
S31508005058EEE7FEF72BFE4023024601210148FEF73C
S315080050685BFF70BD280B00201C520008E40A0020CC
S3150800507808B5FFF70DFD08BD08B5FFF715FD08BD0E
S3150800508808B5FFF745FD08BD08B5FFF785FD08BD56
S3150800509808B5FFF7CFFD08BD08B5FFF757FD034666
S315080050A808B9184608BDFFF7A3FD0346F9E772B61F
S315080050B8704762B670470000F8B500BFF8BC08BC70
S315080050C89E467047F8B500BFF8BC08BC9E467047B0
S315080050D80000002000000000000000000102030490
S315080050E80607080900000000010203044465666112
S315080050F8756C740057696E5553422042756C6B205F
S31508005108496E746572666163650000004F70656E66
S31508005118424C5420557365720000000057696E5555
S3150800512853422042756C6B204465766963650000B6
S315080051386D61696E2E630000757362645F636F6ED6
S31508005148662E63004F70656E424C54002E2E2F2E25
S315080051582E2F2E2E2F536F757263652F41524D438E
S315080051684D375F53544D333246372F7273323332C5
S315080051782E6300002E2E2F2E2E2F2E2E2F536F75B0
S315080051887263652F41524D434D375F53544D333241
S3150800519846372F63616E2E6300000000050206027B
S315080051A8060307030803090309040A040B040C0485
S315080051B80C050D050E050F050F0610061007100835
S315080051C800800008008000000100000000000108B7
S315080051D8008000000200000000800108008000002E
S315080051E80300000000000208000002000400000096
S315080051F80000040800000400050000000000080874
S31508005208000004000600000000000C080000040066
S31508005218070000002E2E2F2E2E2F2E2E2F536F7599
S315080052287263652F41524D434D375F53544D3332A0
S3110800523846372F7573622E6300000000D5
S30D0800524451020008ED01000803
S3090800524CC90100087E
S3150800525000000000EC02002054030020BC030020DC
S315080052600000000000000000000000000000000030
S315080052700000000000000000000000000000000020
S315080052800000000000000000000000000000000010
S315080052900000000000000000000000000000000000
S315080052A000000000000000000000000000000000F0
S315080052B000000000000000000000000000000000E0
S315080052C000000000000000000000000000000000D0
S315080052D000000000000000000000000000000000C0
S315080052E000000000000000000000000000000000B0
S315080052F0000000000000000001000000000000009F
S315080053000E33CDAB34126DE6ECDE05000B00000063
S31508005310000000000000000000000000000000007F
S31508005320000000000000000000000000000000006F
S31508005330000000000000000000000000000000005F
S31508005340000000000000000000000000000000004F
S315080056700000000000000000080E00200024F400CE
S315080056800100000010000000313700083D3700080F
S31508005690ED370008C9370008B5370008093800088B
S315080056A02D3800081201000200000040501DAC60B1
S315080056B00002010203010000040309041A030000A2
S315080056C000000000000000000000000000000000CC
S315080056D00000000000000000853C00086D3C000842
S315080056E00D3C00080000000000000000F53B000823
S315080056F0FF3B0008E13B0008000000000000000036
S3150800570000000000C93B000800000000D53B000867
S3150800571009022000010100C0320904000002FF004E
S315080057200000070581024000FF070501024000FF4F
S311080057300A060002000000400100040008
S70508000335BA
